:020000040800F2
:10000000C03E00208D01000805010008070100081E
:10001000090100080B0100080000000000000000BA
:100020000000000000000000000000000F010008B8
:10003000110100080000000013010008150100086C
:1000400000000000000000000000000000000000B0
:1000500000000000000000000000000000000000A0
:100060000000000000000000000000000000000090
:100070000000000000000000000000000000000080
:100080000000000000000000000000000000000070
:100090000000000000000000000000000000000060
:1000A0000000000000000000000000000000000050
:1000B0000000000000000000000000000000000040
:1000C0000000000000000000000000000000000030
:1000D0000000000000000000000000000000000020
:1000E0000000000000000000000000000000000010
:1000F0000000000000000000000000000000000000
:10010000640D0008FEE7FEE7FEE7FEE7FEE7FEE718
:10011000FEE7FEE7FEE72020174D01202968014396
:100120002960361F37602F4600B500BF3D680220AA
:100130000540FBD01120114908601148786000206B
:10014000F862104839680143396000BF3D680E48C5
:100150000540FBD03D1D0C3E032131600221716042
:10016000B7602F4600F0A4FA7D680C200540082DEA
:10017000FAD180CE00BD01BC001002400020024038
:1001800000801004000000010000000200B500BF64
:10019000104D85F30888104D85F30988022585F3F5
:1001A0001488BFF36F8F0D4E0D4883460D490E48DE
:1001B0000D6805430D600D490D480D6885430D60C0
:1001C000FFF7AAFF0B48056801200543A847DFE7B2
:1001D00000BD0000C03E0020403F0020B43F002092
:1001E000C03F00201410024014007E00281002407E
:1001F00000007E000001000802CE0124E4077346DF
:100200005B1E1A680919781A07B480CE7046001D63
:100210000047000002CEB942EFD180CE01217046E6
:1002200088430268104700000120384380CE004711
:100230007047202080CE704703CE002200238142E9
:1002400000DB0122B94200DC012300271A4200D062
:10025000FF4370473A4603CE0027121A091A91420B
:1002600000D2FF43704700003846316840B40A04AA
:10027000120C0B0C0404240C050C164666431F4696
:100280006F4318466043010C000436184F4128465E
:100290005043010C000436184F41354640BC3560D0
:1002A0007047202031684F43361D704735687D40C8
:1002B00000B520B4002F00D57F423568002D00D551
:1002C0006D423560FFF7D0FF20BC002D01D500F056
:1002D000C9F800BD01CE31682024002249184041F0
:1002E00013465341C01B5B4101D0491C00E0C019BB
:1002F000641EF3D10F4630607047202000B580B4F3
:1003000035687D4020B480B480CE00F0C1F8009DF7
:10031000002D00D56D42361F37602F46FFF7DAFFFC
:100320001548074020BC002D01D4002501E001251F
:100330006D42002DEFF3008001B43068376007464E
:1003400001BC80F3008800D57F4220BC002DEFF374
:10035000008001B430683760074601BC80F3008834
:1003600008D57F423068002804D07F1E009D306889
:100370002D1A356001B000BDFFFFFF7F00B530686A
:1003800001B480B480CE00F083F8009D002D00D52C
:100390006D42361F37602F46FFF79CFF20BC009C44
:1003A0006C40002C00D57F4220BC002DEFF3008074
:1003B00001B430683760074601BC80F3008800D57F
:1003C0007F4230683760074600BD202000B580B40A
:1003D0003168CF1720BC361F37602F46FFF7CEFF9E
:1003E00000BD202000B580B43168CF1720BC361F77
:1003F00037602F46FFF7C2FF361D00BD361F0021B4
:10040000316000B5FFF766FF361D00BD00B5FFF790
:10041000DDFF80CE00BD202000B580B480CEFFF788
:1004200045FF20BC361F37602F46FFF7A7FF00BDF2
:1004300000B5FFF7F1FF361D00BD202000B5FFF726
:100440009DFF361D00BD000007CE80184F41361FAE
:100450003060704707CE101AB9410F46361F306022
:1004600070470000306800214042B9410F463060BB
:10047000704700003F1C80CE00D57F4270470000CF
:100480003F1C80CEEED47047002F00D57F427047CE
:100490003F1CE7D470470000B800002801DC80CE84
:1004A00070473758011F72583250081CFAD1361D58
:1004B000704700003B1C83CE00D17047021C0A43EA
:1004C0001A430324144006D10A680260091D001D66
:1004D0001B1FF9D170470A780270491C401C5B1E33
:1004E000F9D170473B1C83CE00D17047C018C918A2
:1004F000021C0A431A430324144006D1091F001F9B
:100500000A6802601B1FF9D17047491E401E0A7815
:1005100002705B1EF9D170473A1C83CE002803D0CD
:100520000A70491C401EFBD170472020361F3760DF
:10053000002700B5FFF7F0FF00BD000003CE3F1C11
:1005400007D002780B78401C491C9A4201D17F1ECB
:10055000F7D102D101277F4200E000277047000059
:10056000361F3760009F7F1E3978C919091D032285
:100570009143491C0091704700B5FFF7F1FF00BDA2
:1005800000B5FFF7EDFF7D1C3F78361F356000BDDD
:100590000120074380B480CE70470000361F3760CB
:1005A00080BC012087437047361F3760009F0120C1
:1005B00087437047361F37607046401E076800BD8E
:1005C000361F37607046401E076800BD361F376013
:1005D0007046401E07683F6800BD361F3760704692
:1005E000401E07685F4400BD70477046401E0068AB
:1005F00001680122114308BC9E460847361F376038
:10060000202700B500F0A4F900BD2020002F00DC59
:100610000027361F3760002700B500BFFFF7FAFD3F
:1006200033060008FFF7EAFF0098401C0090F9D756
:1006300003B000BD0F200740092F00B500DDFF1DEE
:10064000303700F085F900BD3D09361F37602F4671
:1006500000B5FFF7EFFFFFF7EDFF00BD3D0B361FC5
:1006600037602F4600B5FFF7E5FF3D0A361F3760BC
:100670002F46FFF7DFFF3D09361F37602F46FFF794
:10068000D9FFFFF7D7FF00BD3D0C361F37602F465F
:1006900000B5FFF7E3FFFFF7E1FF00BD00B5FFF78F
:1006A000F3FF00BD00B500BFFFF79FFF0000002073
:1006B0003D683068C4432C40706804433C60B768B0
:1006C0000C36704700B500BF3D68002D04D03D6872
:1006D0007C682C600837F7E780CE00BD1A4D2C46A9
:1006E0003034103E0321316000217160B560F76045
:1006F000274600B5FFF7DCFF1448796901437961AB
:100700001248B96A8143B9621148B9690143B961B4
:100710000F48F9688143F9600E4801B4009F3F1CFF
:10072000083E0D4931600D497160FFF7C1FF20BCE3
:1007300024350C3E0A4931600A497160B7602F4682
:10074000FFF7B6FF00BD00000010024000000200ED
:10075000004000000000004800003C0000002800AD
:10076000F00F000010010000FF69202007407047D3
:1007700000B500BFFD6920200540002D02D1FFF724
:1007800091FFF7E77F6AFF20074000BD00B500BF7B
:10079000FD6980200540002D02D1FFF783FFF7E7B8
:1007A0003068B8627768083600BD2020706831680C
:1007B0004518706877600746356000B5FFF72AFD79
:1007C000E1070008009D019805442D78083E35603A
:1007D0007760FFF7DBFF0098401C0090F2D703B072
:1007E00080CE00BD083E0D213160776000B5FFF777
:1007F000CDFF361F0A213160FFF7C8FF00BD202062
:100800007047202000203860002078600020B86009
:100810003068F8600C2038600D2038607768083642
:100820007047202000B5FFF759FF083E03493160AB
:100830007760034FFFF7E6FF00BD0000A101000055
:1008400000380140361F3760024F00B5FFF78CFFBC
:1008500000BD000000380140361F3760024F00B570
:10086000FFF786FF00BD000000380140361F3760EB
:10087000024F00B5FFF78AFF00BD000000380140BD
:10088000361F3760024F00B5FFF790FF00BD000034
:1008900000380140361F3760024F00B5FFF7A2FF56
:1008A00000BD00000038014000B500BFFFF782FE28
:1008B000B408000858080008440800086C0800083C
:1008C000800800089408000800B500BFFFF772FE1A
:1008D000B408000800B5FFF7A5FF00BD00B500BFD4
:1008E000FFF77BFE0000000000B500BFFFF775FEBC
:1008F0001800000000B500BFFFF76FFE1C000000ED
:1009000000B500BFFFF769FE2000000000B500BF82
:10091000FFF763FE2400000000B500BFFFF75DFE97
:100920002800000000B500BFFFF757FE2C000000B4
:100930005D46ED6A2D6800B501200543A84700BD5E
:100940005D46ED6A6D6800B501200543A84700BD0E
:100950005D4624352978491C29705D46AD6AAD682D
:1009600000B501200543A84700BD20205D46243581
:100970002978C91929705D46AD6AED6800B5012076
:100980000543A84700BD20205D462435002028707F
:100990005D46AD6A2D6900B501200543A84700BD3D
:1009A00000B5FFF7DDFD7D1C3F78361F3560FFF792
:1009B000DDFF00BD361F3760004F01E0DC0D000891
:1009C00000B500BF3D68002D0FD03D460C353C689A
:1009D0007B680C3E33607560B7602746FFF76AFDA1
:1009E0003D68ED190C352F46ECE780CE00BD202088
:1009F00000B5FFF731FFFE2F80CE01D000F07EF969
:100A000000BD202000B5FFF731FFFFF7F1FF00BD6B
:100A100000B5FFF721FF361F3760FE27FFF726FFDF
:100A200000BD2020083E0021316077600D4F00B5E9
:100A3000FFF750FCFFF71AFF083E00213160776096
:100A4000094FFFF747FCFFF711FF083E0021316017
:100A50007760064FFFF73EFCFFF708FFFFF706FF42
:100A600000BD0000000000010000010000010000C6
:100A700000B5FFF7CDFF3F06FFF7CAFF3F04306820
:100A80003F18361DFFF7C4FF3F0230683F18361D80
:100A9000FFF7BEFF30683F18361D00BD5D46AD69EB
:100AA000361F37602F46361F376037463168CF1BF9
:100AB0003F1FBF10361D704700B5FFF7EFFF361F11
:100AC0003760FFF7AFFF002F00D180CE17D07F1E19
:100AD000361F0021316000BFFFF78EFBFF0A0008C0
:100AE000009D01980544361F37602F46BF00F75917
:100AF000FFF798FF0098401E0090F1D703B000BDAB
:100B00005D46AD69361F37602F463E1C80CE00B56E
:100B1000FFF7AEFF361F3760002700BFFFF77AFBF5
:100B2000330B0008FFF7A4FF0098401C0090F9D792
:100B300003B000BD361F3760842700B5FFF762FFA2
:100B4000FFF796FF00BD2020361F3760812700B5D4
:100B5000FFF758FFFFF78CFF00BD2020361F3760DE
:100B6000822700B5FFF74EFFFFF780FE00BD202073
:100B7000361F3760832700B5FFF744FFFF2007408B
:100B8000361F3760FFF772FE30683F1830683760F5
:100B9000074600BFFFF73EFBB90B0008009D019818
:100BA00005442D78361F37602F46FFF75FFE00980B
:100BB000401C0090F2D703B000BD2020361F3760E4
:100BC0000D2700B5FFF7CAFF361F37600A27FFF76A
:100BD000C5FF00BD00B500BFFFF7ECFCE00B00084F
:100BE000480B0008340B00085C0B0008700B000871
:100BF000BC0B000800B5FFF783FF3D4680CE012007
:100C00000543A847361F3760FF27FFF72FFEFFF782
:100C100053FF00BD00B5FFF72BFF3F88FFF702FF32
:100C200000BD202000B5FFF723FFFFF721FF30684C
:100C300038807768083600BD00B5FFF719FF3F78A8
:100C4000FFF714FE00BD202000B5FFF711FFFFF7EE
:100C50000FFF306838707768083600BD00B5FFF7C1
:100C600007FF3F68FFF7DEFE00BD202000B5FFF75D
:100C7000FFFEFFF7FDFE306838607768083600BD7C
:100C800000B5FFF7F5FEFFF7F3FE30683F18306858
:100C900037600746FFF7BEFAB50C0008FFF7B8FE4D
:100CA000009D019805442F7080CE0098401C009054
:100CB000F4D703B000BD2020361F3760FD2700B5F4
:100CC000FFF7D4FD00F01AF800BD0000F40B000897
:100CD000700A0008240A0008000B0008B80A00087F
:100CE000140C0008240C0008380C0008480C0008FC
:100CF0005C0C00086C0C0008800C00085D46ED6977
:100D000000B5AD46FFF7A8FD7F1E0B2F01D9FD27CB
:100D100022E0361F3760FE27FFF7A8FDBF0010480E
:100D20003F183F683D4680CE01200543A847FFF7A6
:100D30005FFEFFF7B3FE1E2F80CE0AD95D46AD6978
:100D4000361F37602F463E1C80CE361F3760FC278B
:100D500002E0361F3760FF27FFF788FDD2E700BDAE
:100D6000CC0C000800B5FFF719FC6F465D46EF613B
:100D700080CE361F376037465D46AF615F46084814
:100D8000B8625F460648F86280CEFFF713FEFFF7B1
:100D9000A1FD5D460A202862FFF7B0FF00BD0000FC
:100DA000E00B000800B5FFF7FBFD0E4D504520534A
:100DB000544D33324630373220000000FFF7F0FD4B
:100DC0000A556D62696C6963616C2000FFF7E8FD8C
:100DD00005466F727468000000BD0000040000004A
:100DE00000000020000000003002000800000000A9
:00000001FF
